:100000000C9498030C94C0030C94C0030C94C0038C
:100010000C94C0030C94C0030C94C0030C94C00354
:100020000C94C0030C94C0030C9466090C94D5097D
:100030000C94C0030C94C0030C94C0030C94C00334
:100040000C94C0030C94C0030C94C0030C94C00324
:100050000C94C0030C94C0030C94C0030C94070CC4
:100060000C94C0030C94C0030C94C0030C94C00304
:100070000C94C0030C94C0030C94C0030C94C003F4
:100080000C94C0030C94C0030C94C0030C94C003E4
:100090000C94C0030C94C0030C94C0030C94C003D4
:1000A0000C94C0030C94C0030C94C0030000000027
:1000B000003E5B4F5B3E3E6B4F6B3E1C3E7C3E1CEE
:1000C000183C7E3C181C577D571C1C5E7F5E1C0034
:1000D000183C1800FFE7C3E7FF0018241800FFE7EB
:1000E000DBE7FF30483A060E2629792926407F05AE
:1000F0000507407F05253F5A3CE73C5A7F3E1C1CC4
:1001000008081C1C3E7F14227F22145F5F005F5F83
:1001100006097F017F006689956A6060606060946F
:10012000A2FFA29408047E040810207E2010080874
:100130002A1C08081C2A08081E101010100C1E0C7F
:100140001E0C30383E3830060E3E0E060000000011
:100150000000005F00000007000700147F147F14F8
:10016000242A7F2A1223130864623649562050003D
:1001700008070300001C2241000041221C002A1C29
:100180007F1C2A08083E0808008070300008080814
:100190000808000060600020100804023E51494534
:1001A0003E00427F400072494949462141494D3352
:1001B0001814127F1027454545393C4A49493141B9
:1001C000211109073649494936464949291E000087
:1001D00014000000403400000008142241141414DC
:1001E0001414004122140802015909063E415D59C8
:1001F0004E7C1211127C7F494949363E41414122D1
:100200007F4141413E7F494949417F090909013EFA
:10021000414151737F0808087F00417F4100204021
:10022000413F017F081422417F404040407F021C33
:10023000027F7F0408107F3E4141413E7F0909094A
:10024000063E4151215E7F09192946264949493216
:1002500003017F01033F4040403F1F2040201F3FDC
:100260004038403F63140814630304780403615961
:10027000494D43007F4141410204081020004141A3
:10028000417F04020102044040404040000307084F
:100290000020545478407F2844443838444444284B
:1002A000384444287F385454541800087E090218F2
:1002B000A4A49C787F0804047800447D400020407A
:1002C000403D007F1028440000417F40007C0478BE
:1002D00004787C080404783844444438FC18242406
:1002E0001818242418FC7C08040408485454542486
:1002F00004043F44243C4040207C1C2040201C3C03
:100300004030403C44281028444C9090907C4464F9
:10031000544C44000836410000007700000041368C
:10032000080002010204023C2623263C1EA1A16112
:10033000123A4040207A3854545559215555794144
:100340002154547841215554784020545579400C1B
:100350001E527212395555555939545454593955FC
:100360005454580000457C410002457D420001453F
:100370007C40F0292429F0F0282528F07C545545AC
:10038000002054547C547C0A097F4932494949323F
:100390003248484832324A4848303A4141217A3A54
:1003A00042402078009DA0A07D39444444393D401E
:1003B00040403D3C24FF2424487E4943662B2FFCCB
:1003C0002F2BFF0929F620C0887E09032054547979
:1003D000410000447D413048484A32384040227A4A
:1003E000007A0A0A727D0D19317D2629292F2826C7
:1003F0002929292630484D402038080808080808CF
:100400000808382F10C8ACBA2F102834FA00007B27
:10041000000008142A142222142A1408950022002D
:1004200095AA005500AAAA55AA55AA000000FF00E7
:10043000101010FF00141414FF001010FF00FF1024
:1004400010F010F0141414FC001414F700FF000056
:10045000FF00FF1414F404FC141417101F10101FD5
:10046000101F1414141F00101010F0000000001FC3
:10047000101010101F10101010F010000000FF10CE
:100480001010101010101010FF10000000FF1400CA
:1004900000FF00FF00001F10170000FC04F41414FC
:1004A0001710171414F404F40000FF00F7141414C8
:1004B00014141414F700F7141414171410101F1048
:1004C0001F141414F4141010F010F000001F101F6B
:1004D0000000001F14000000FC140000F010F010D9
:1004E00010FF10FF141414FF141010101F00000050
:1004F00000F010FFFFFFFFFFF0F0F0F0F0FFFFFF54
:100500000000000000FFFF0F0F0F0F0F38444438AA
:10051000447C2A2A3E147E02020606027E027E02E5
:1005200063554941633844443C04407E201E200604
:10053000027E020299A5E7A5991C2A492A1C4C7241
:1005400001724C304A4D4D303048784830BC625AC8
:10055000463D3E494949007E0101017E2A2A2A2A58
:100560002A44445F444440514A444040444A514034
:100570000000FF0103E080FF000008086B6B0836F5
:1005800012362436060F090F060000181800000066
:100590001010003040FF0101001F01011E00191D55
:1005A0001712003C3C3C3C0000000000F0F89C8E20
:1005B0008783878E9CF8F00000FEFF03030303038C
:1005C000070EFCF80000FEFF0303030303070EFC05
:1005D000F80000FFFF00000000000000FFFF000027
:1005E000FEFF8383838383C7EE7C380000F8FC0E14
:1005F00007030303070EFCF800003F7FE0C0808084
:10060000C0E07F3FFFFF01010101010101FFFF0089
:1006100000FFFF0C0C0C0C1C3E77E3C100007FFFB9
:10062000C0C0C0C0C0E0703F1F00001F3F70E0C0EE
:10063000C0C0E0703F1F00007FFFC1C1C1C1C1E366
:10064000773E1C00001F3F70E0C0C0C0E0703F1F3D
:10065000000000000001FFFF01000000D5F08D1434
:10066000A1C881CFD9F1AF20003E09093F3F3E002C
:10067000003F3F2020202000003F060C063F3F00A7
:10068000001E3F21213F1E00001227253D3D18007E
:100690000001013F3F01010000000000003F3F0951
:1006A000090F0600001E3F21213F1E00003F060CDF
:1006B000183F3F00001E3F21293B3A080B00020271
:1006C00002000009040000010202000005240010DD
:1006D0000105240101010424020605240600010786
:1006E00005810310004009040100020A0000000710
:1006F00005020240000007058302400000040309D0
:100700000412010002EF0201404123378000010181
:1007100002030141726475696E6F204C4C430041C5
:10072000726475696E6F204D6963726F0000C90C49
:1007300011241FBECFEFDAE0DEBFCDBF11E0A0E095
:10074000B1E0E6ECFAE202C005900D92AA38B107DA
:10075000D9F726E0AAE8B1E001C01D92A531B207A1
:10076000E1F713E0C8E9D3E004C02197FE010E943D
:100770005615C739D107C9F70E94FA0C0C946115B8
:100780000C940000480F592F511D1416150684F5BE
:10079000803891056CF597FF02C090E080E0413809
:1007A000510514F040E850E0481BFB01E770FF27BB
:1007B00021E001C0220FEA95EAF777FF02C0695FE6
:1007C0007F4FFB0133E0F595E7953A95E1F7F69514
:1007D000FE2FEE27F795E795E80FF91FE255FE4F3C
:1007E000415030F08191DF011197822B8C93F8CF2B
:1007F000089580E0EEEAF1E081118FEF002481930B
:100800008193819381930394D1F70895EEEAF1E007
:10081000A0E0B8E000800EBC8111012C1197A0FD72
:10082000FDCF0192B9F70DB408958F929F92AF92C8
:10083000BF92CF92DF92EF92FF920F931F93CF93CD
:10084000DF93FC01E20FF11DF7FD88C080349105B4
:100850000CF084C0DC0197FF04C0AA27BB27A81BAB
:10086000B90BA770BB27FC0197FD379633E0F595D0
:10087000E7953A95E1F797FF07C0319788E090E058
:10088000EC01CA1BDB0BDE01E22EE694E694E69453
:10089000F12C277019F0DFEFED1AFD0A50E0CF01BF
:1008A000EB018F011695102F00271795079502551C
:1008B0001E4F97012E0F3F1F68E070E05B01AA1AE0
:1008C000BB0A8217930709F449C08830910509F4DF
:1008D00045C08F3FEFEF9E07C4F170E060E0780104
:1008E000F0E8EF0EF11C8F3F9807A9F1FE01E60F2B
:1008F000F71FE4916801C60ED71EF0E04F010A2EE3
:1009000001C0880C0A94EAF7F60194888928848A41
:100910001097B1F08730910599F0FB01EC0FFD1FA6
:10092000E4916701C60ED71EF0E04F010A2C02C009
:10093000959487940A94E2F7F60194888928848A2A
:100940006F5F7F4F6417750774F20196C40FD51F50
:1009500000581F4FB6CF109799F3DFCFDF91CF919B
:100960001F910F91FF90EF90DF90CF90BF90AF90CD
:100970009F908F900895FC018091AD01882311F123
:100980003FB7F89482E08093E9002091F200822F33
:1009900090E01816190614F481E090E0882339F0ED
:1009A000289A44E64093AC014091F1004083222311
:1009B00039F02091F200211103C02BE62093E800CA
:1009C0003FBF08958FEF9FEF08952FB7F89483E00E
:1009D0008093E9009091E800892F807295FF04C010
:1009E0009091F20080E4891B2FBF08958091A401AB
:1009F00081110DC082E08093A00184E08093A10169
:100A00001092A3011092A20181E08093A40180EAD8
:100A100091E00895CF93DF931F92CDB7DEB769833E
:100A2000DC01ED91FC910280F381E02D41E050E08A
:100A3000BE016F5F7F4F09950F90DF91CF910895B1
:100A400083E08093E9008091F200882319F08AE323
:100A50008093E80008950E94E50490E00895CF9304
:100A6000DF931F92CDB7DEB7FC018485958597FD96
:100A700008C02FEF3FEF358724870F90DF91CF918C
:100A80000895CE0101960E94BB04019719F4898153
:100A900090E0F3CF8FEF9FEFF0CF0F931F93CF93A3
:100AA000DF931F92CDB7DEB78C01FC01848595855D
:100AB00097FF0BC0CE0101960E94BB04019771F411
:100AC000898190E0F80195878487F8018485958570
:100AD0000F90DF91CF911F910F9108958FEF9FEFAE
:100AE000F1CFFC018485958597FD0BC09FB7F894E5
:100AF00082E08093E9008091F2009FBF90E0019630
:100B000008959FB7F89482E08093E9008091F20005
:100B10009FBF90E0089540919A0150919B012091D0
:100B200098013091990142175307B4F49091E8006D
:100B30009570E1F39091E80092FD19C08093F10067
:100B400080919A0190919B0101968F739927892B2F
:100B500019F48EEF8093E80080919A0190919B01A7
:100B6000019690939B0180939A0181E0089580E023
:100B70000895DF92EF92FF920F931F93CF93DF932D
:100B8000D82E8A01EB017B01E40EF51ECE15DF05A0
:100B900059F0D7FE12C0FE0184910E948B05219668
:100BA0008111F4CF0FEF1FEFC801DF91CF911F919B
:100BB0000F91FF90EF90DF9008958881EECF0F9313
:100BC0001F93CF93DF931F92CDB7DEB782E0898367
:100BD00042E450E06BEB76E080E80E94B9050E94A9
:100BE000F604DC0112960D911C910115110589F096
:100BF000D801ED91FC910280F381E02DBE016F5F81
:100C00007F4FC801099597FD04C0F8010085118543
:100C1000ECCF89810F90DF91CF911F910F910895B3
:100C2000615030F02091F100FC0120830196F8CF53
:100C3000289A84E68093AC010895AF92BF92CF9238
:100C4000DF92EF92FF920F931F93CF93DF936C018C
:100C50007B018B01040F151FEB015E01AE18BF086D
:100C6000C017D10759F06991D601ED91FC9101901F
:100C7000F081E02DC6010995892B79F7C501DF9137
:100C8000CF911F910F91FF90EF90DF90CF90BF9089
:100C9000AF9008953FB7F89480918B0190918C01AB
:100CA000A0918D01B0918E0126B5A89B05C02F3F64
:100CB00019F00196A11DB11D3FBFBA2FA92F982F82
:100CC0008827BC01CD01620F711D811D911D42E07D
:100CD000660F771F881F991F4A95D1F708958F9245
:100CE0009F92AF92BF92CF92DF92EF92FF926B01F1
:100CF0007C010E944A064B015C01C114D104E1044D
:100D0000F104B9F00E944A06681979098A099B0919
:100D1000683E73408105910580F321E0C21AD10835
:100D2000E108F10888EE880E83E0981EA11CB11C32
:100D3000E4CFFF90EF90DF90CF90BF90AF909F9067
:100D40008F9008958F929F92AF92BF92CF92DF9231
:100D5000EF92FF920F931F93CF93DF936C017B0170
:100D60008A0180912D01882309F45CC08091AD0136
:100D7000882309F457C080919F0180FF05C08091AE
:100D8000E00082608093E000E801B12C8AEFA82E99
:100D900093E0892E2AE3922E209711F4BB20D9F1FB
:100DA0000E94E50481110AC0AA94AA20D9F161E049
:100DB00070E080E090E00E946F06EECF8C171D0679
:100DC00011F00CF08C2F9FB7F8948092E9002091DD
:100DD000E80025FD02C09FBFDFCF282F30E0C21BF7
:100DE000D30BF701815020F041914093F100FACFED
:100DF000E20EF31EBB2021F09092E800B12CEBCF65
:100E00008091E80085FDE7CF9092E800BB24B39481
:100E1000209709F3F3CF5D9A84E680939E01101624
:100E200011063CF081E090E0F6019383828310E0AC
:100E300000E0C801DF91CF911F910F91FF90EF90DB
:100E4000DF90CF90BF90AF909F908F9008952D9A94
:100E50000895BC0190E080E00C946F068FB18095FE
:100E6000807F669B88601C9B8460089520E191E0F0
:100E700061FD94E060FD990F62FD9295687F269F69
:100E8000D0011124A80FA255BE4F8C9140FF03C082
:100E9000892B8C93089590958923FBCFEF92FF9235
:100EA0000F931F93CF93DF937C018B01040F111DD0
:100EB000EB0177FF02C0D0E0C0E0C80101341105AA
:100EC00014F080E490E0C817D9075CF480E8E816D5
:100ED000F10428F441E0BE01C7010E9436072196C3
:100EE000ECCFDF91CF911F910F91FF90EF9008957C
:100EF000EF92FF920F931F93CF93DF937C018B01AF
:100F0000C42FD22F6034710510F40E94C203B801BF
:100F10006D0F711D615071096034710520F44C2F03
:100F2000C7010E94C2034D2FB801C7010E944E079E
:100F3000C7018C0F911D4D2FB8010197DF91CF9103
:100F40001F910F91FF90EF900C944E072F923F92BC
:100F50004F925F926F927F928F929F92AF92BF92C9
:100F6000CF92DF92EF92FF920F931F93CF93DF9375
:100F7000CDB7DEB728970FB6F894DEBF0FBECDBF52
:100F80009E838D836A3061F5DC0155968C91B8E0C3
:100F90008B9F90011124ED81FE8181899289820FBE
:100FA000931F928B818B108A178681E090E02896A0
:100FB0000FB6F894DEBF0FBECDBFDF91CF911F916A
:100FC0000F91FF90EF90DF90CF90BF90AF909F90E8
:100FD0008F907F906F905F904F903F902F900895EB
:100FE0006D3019F32D813E8138872F83D9011F96EB
:100FF0000D911C915097003811050CF07CC0519652
:10100000AD90BC90B0E4AB16B1040CF074C0F90123
:10101000258825E0C801229E800D911D11241816F7
:1010200019060CF068C0622C712CC30133E0880FE4
:10103000991F3A95E1F78A0D9B1D181619060CF0B9
:101040005AC0F489FB83AF81B8855396BC91BC83A9
:10105000629FB0011124FB01E455FF4F2F0119825B
:10106000F2018491F981F53009F480E0450128E02E
:101070002A83A82FB0E0BE83AD833C8080FF3B80F5
:10108000311004C0BB81EC81BE17F9F078018E2DC0
:10109000801B8215D0F4D12CC12CC21490F4F0E83E
:1010A000EF16F10450F4B601680D791D6034710536
:1010B00020F4432DC7010E9436072FEFC21AD20A2F
:1010C000ECCF3FEFE31AF30AE2CF8D819E81959535
:1010D00087959A8191509A83860C971C9111C9CF5C
:1010E000A981AF5FA983BFEF4B1A5B0A060D171DDD
:1010F000A63009F0B5CFEF81F8852589422F50E061
:1011000087859089F6E02F9F800D911D1124AF8176
:10111000B88550969C938E931F9756962C91569710
:10112000222309F442CF6AEF64039001659F300DDA
:10113000112420583F4F281739070CF036CFED9176
:10114000FC9111970190F081E02D6AE0CD010995A5
:101150002CCF0895089590E080E008958F929F929B
:10116000AF92BF920F931F93CF93DF93CDB7DEB7AC
:10117000A1970FB6F894DEBF0FBECDBF19A24230C3
:1011800008F44AE08E010F5D1F4F842E912CB12C84
:10119000A12CA50194010E944513E62FB901CA01B3
:1011A000EA3044F5E05DD801EE938D01232B242B2A
:1011B000252B79F790E080E0109769F0FD01019010
:1011C0000020E9F73197AF014A1B5B0BBD018EEFA1
:1011D00095E00E941D06A1960FB6F894DEBF0FBEE3
:1011E000CDBFDF91CF911F910F91BF90AF909F9096
:1011F0008F900895E95CD7CFFC0101900020E9F7BA
:101200003197AF01481B590BBC018EEF95E00C9450
:101210001D06CF92DF92EF92FF92CF93DF936C0186
:10122000990FEE08FF08F7FE19C06DE28EEF95E00A
:101230000E94A607EC0166277727CB016C197D0970
:101240008E099F094AE00E94AE088C0F9D1FDF9116
:10125000CF91FF90EF90DF90CF9008954AE0C701C3
:10126000B601DF91CF91FF90EF90DF90CF900C947B
:10127000AE08CF92DF92EF92FF92CF93DF93EC0113
:101280000E94A5122AE2C22ED12CE12CF12CA7013A
:1012900096010E9413136D5F7F4F8F4F9F4F69839D
:1012A0000E94A512A70196010E9413136D5F7F4F44
:1012B0008F4F9F4F6B83DF91CF91FF90EF90DF9027
:1012C000CF9008950C94FD120E945C151F920F920E
:1012D0000FB60F9211248F939F938091E10090910C
:1012E000E100937F9093E10083FF0FC01092E9002B
:1012F00091E09093EB001092EC0092E39093ED005C
:101300001092AD0198E09093F00082FF22C093E02C
:101310009093E9009091F200992319F09AE3909349
:10132000E80090919E01992341F090919E01915087
:1013300090939E01911101C05D989091AC01992309
:1013400041F09091AC0191509093AC01911101C08A
:10135000289884FF18C08091E2008E7E816080937F
:10136000E2008091E1008F7E8093E10080919F01F7
:101370008E7E806180939F019F918F910F900FBE11
:101380000F901F90189580FFF7CF8091E2008E7E1E
:1013900080618093E2008091E1008E7E8093E10085
:1013A00080919F018E7E8160E5CF1F920F920FB6D4
:1013B0000F921124CF92DF92EF92FF920F931F931F
:1013C0002F933F934F935F936F937F938F939F934D
:1013D000AF93BF93EF93FF93CF93DF93CDB7DEB778
:1013E0006C97DEBFCDBF1092E9008091E80083FFCB
:1013F00025C068E0CE0145960E94100682EF8093DA
:10140000E8008D8987FF39C09091E80090FFFCCFFC
:10141000982F907609F034C19E894F89588D2F8975
:10142000F88C911131C0803861F580919D018093D5
:10143000F1001092F1008EEF8093E8006C960FB6E9
:10144000F894DEBF0FBECDBFDF91CF91FF91EF913A
:10145000BF91AF919F918F917F916F915F914F91CC
:101460003F912F911F910F91FF90EF90DF90CF90C0
:101470000F900FBE0F901F9018959EEF9093E8006D
:10148000C7CF1092F100D5CF913059F48111D3CF4D
:101490004130510581F680919D018D7F80939D01A2
:1014A000CACF933049F48111C6CF4130510519F6A6
:1014B00080919D018260F2CF953041F48091E800E7
:1014C00080FFFCCF20682093E300B5CF963009F071
:1014D000A9C00B8D1C8D22E01092E90010929B0197
:1014E00010929A01F2122EC0109299011092980156
:1014F0000E94DF051F8299E09983FA8291E09E8322
:1015000090EA98879AEF998720919A0130919B01F0
:10151000275F3F4F3C832B838D831092E90010920D
:101520009B0110929A01109399010093980149E050
:1015300050E0BE016F5F7F4F80E00E94B9050E94BE
:10154000DF0579CF10939901009398010E94F6046A
:10155000DC0112960D911C910115110509F451C180
:10156000D801ED91FC910480F581E02DBE016B5E08
:101570007F4FC8010995009709F03EC1F801008529
:101580001185EACFF3E0FF120EC08F89882309F49A
:1015900040C0823061F440E86DE08FE197E00E9446
:1015A000510C811148CF81E28093EB0047CF81300D
:1015B00029F440E86BE083E197E0F1CF833099F7BD
:1015C0000E94F604DC011296ED90FC908E010F5FF4
:1015D0001F4F6801E114F10479F0D701ED91FC91FE
:1015E0000680F781E02DB801C7010995080F111D8C
:1015F000F701E084F184EECFD8011C92F60101904E
:101600000020E9F73197BF016C197D0940E0C60160
:10161000C6CF6DEF76E0FB01449150E080E80E9478
:10162000B90509CF973009F4BECF983021F481E095
:101630008093F10000CF993009F0FDCE837009F05E
:10164000B2CFE3E3F1E081E031E096E321912223A0
:1016500071F08093E9003093EB00DF0111972C913A
:101660002093EC009093ED008F5F873079F78EE741
:101670008093EA001092EA008F898093AD01DBCE5F
:101680008B8D9C8D1092E90010929B0110929A0113
:101690009093990180939801898D811192C08E89D0
:1016A0009D89913A49F4813209F07DCF47E050E0BD
:1016B00066E271E080E0B3CF913209F074CF8332FB
:1016C00069F48F89988DB0E0A0E080932201909317
:1016D0002301A0932401B0932501ADCE803269F49B
:1016E0008091E80082FFFCCF67E086E291E00E94F3
:1016F00010068BEF8093E8009ECE823209F09BCEDD
:101700008F8980932D01EEEFFFE7859194918B3FB8
:101710009C4D51F1E0E0F8E0809126019091270185
:10172000A0912801B0912901803B9440A105B10509
:10173000F1F480912D0180FD1AC0EE3F8AE0F80798
:1017400089F587E797E79183808380916000809394
:101750009C0188E19BE00FB6F894A8958093600007
:101760000FBE9093600067CEEEEFFAE0D5CF808198
:1017700091818737974709F05ECEA89580916000E8
:1017800088618093600080919C0180936000EE3FAF
:101790002AE0F20789F08091FE0A9091FF0A918376
:1017A000808349CE808191818737980751F2909349
:1017B000FF0A8093FE0AC5CF1092FF0A1092FE0A1C
:1017C0003ACE0E94F604DC0112960D911C9101158F
:1017D000110509F4E8CED801ED91FC910190F0815A
:1017E000E02DBE016B5E7F4FC8010995811123CEAC
:1017F000F80100851185EBCF181619060CF41BCEE5
:10180000D2CEF1E0FF12BECE61E077E004CF1F92AE
:101810000F920FB60F9211242F933F938F939F93A4
:10182000AF93BF9380918F0190919001A09191010E
:10183000B091920130918A0123E0230F2D3758F5A2
:101840000196A11DB11D20938A0180938F01909371
:101850009001A0939101B093920180918B0190919E
:101860008C01A0918D01B0918E010196A11DB11D39
:1018700080938B0190938C01A0938D01B0938E0186
:10188000BF91AF919F918F913F912F910F900FBE7C
:101890000F901F90189526E8230F0296A11DB11DE9
:1018A000D2CFEF92FF920F931F93CF93DF93F82E37
:1018B000192FE62E042F81E0860F880F0E948B05DA
:1018C00083E00E948B05CF2DD12FEC0EFD2EF11C55
:1018D000CE15DF05B9F007FF13C0FE0184910E9409
:1018E0008B05182F80E00E948B05812321968111A2
:1018F000EFCFDF91CF911F910F91FF90EF9008955F
:101900008881EDCF81E0F5CF0F931F93CF93DF93C5
:101910008C0181E090E00E94620980FF32C08AE081
:1019200090E00E9462099FEF980F9E3F50F522E3DE
:1019300030E0D80150963C932E931F9728E330E077
:1019400052963C932E935197CBE0D0E0D801ED9185
:10195000FC910190F081E02D682FC8010995CE011E
:101960000E9462092196C131D10581F780E00E9471
:10197000060488EE93E0DF91CF911F910F910C94B4
:101980002907DF91CF911F910F91089504970C942F
:10199000840CEEEAF5E01382128288EE93E0A0E078
:1019A000B0E084839583A683B7838DE391E0918330
:1019B00080838FEF9FEF95878487EEEFF5E01382AA
:1019C00012821186128680E183871086178215861F
:1019D0008FE491E0918380838DE591E0958384830A
:1019E000108A1786128A118A81E0838B148A858B6C
:1019F000168A0895CF93DF93CDB7DEB72A970FB637
:101A0000F894DEBF0FBECDBF789484B5826084BDEC
:101A100084B5816084BD85B5826085BD85B58160F2
:101A200085BD80916E00816080936E001092810070
:101A3000809181008260809381008091810081602B
:101A400080938100809180008160809380008091EC
:101A500091008260809391008091910081608093D9
:101A60009100809190008160809390008091C100EE
:101A700084608093C1008091C10082608093C10026
:101A80008091C10081608093C1008091C30081601A
:101A90008093C3008091C00082608093C0008091D9
:101AA000C20081608093C20080917A00846080933C
:101AB0007A0080917A00826080937A0080917A0027
:101AC000816080937A0080917A00806880937A00A8
:101AD0001092AD0110929D0110929F018091D7004C
:101AE00081608093D70080EA8093D80089B58061B7
:101AF00089BD89B5826089BD09B400FEFDCF61E072
:101B000070E080E090E00E946F068091D8008F7CAA
:101B100080618093D8008091E000807F8093E00016
:101B20008091E1008E7E8093E1008DE08093E20061
:101B3000559A209A5D98289881EC80937C0085B115
:101B4000806F85B984B1877E84B984B1876E84B98A
:101B50005E9A5F988AB1806D8AB9769A6E9881B3E1
:101B6000806F81BB899880B38D7080BB80E58CBD10
:101B700081E08DBD85E090E00E9429075F9A85E0B5
:101B800090E00E9429075E985C98ECE5F6E089E613
:101B900096E024912EBD00000DB407FEFDCF3196D6
:101BA0008E179F07B1F75C9A81E88093640080915B
:101BB000650081608093650080E00E9406040E94B9
:101BC0002E0787FF15C05C9885EA8EBD00000DB416
:101BD00007FEFDCF5C9A2E982F982D988091640077
:101BE00080628093640081E083BF889513BEFCCF40
:101BF0000E942E0782FF48C02D980E942E078478ED
:101C00008438E1F40E94270788EC90E00E942907BD
:101C10002F9882E090E00E94FD128F3F29F06FEF35
:101C200082E090E00E94051384EF91E00E94290772
:101C30002F9A0E942E0784788438D9F30E942E07A9
:101C400084718431E1F40E94270788EC90E00E94BF
:101C500029072E9882E090E00E94FD12882329F047
:101C600060E082E090E00E94051384EF91E00E9422
:101C700029072E9A0E942E0784718431D9F388ECAB
:101C800090E00E942907B4CF0E94270782E090E0ED
:101C90000E946209882309F462C03E9A3F9A81E05B
:101CA00090E00E946209182F147081FF0EC011117C
:101CB0002E9880EF9FEF9A8389830E942E0786FFDC
:101CC00051C02E9A2F9A0E94270782E390E00E942B
:101CD00029070E942E078111F8CF86E1809309061B
:101CE0000E94F9031092100610920F0610920E0631
:101CF00010920D0685E0809318018BE780931D01FB
:101D00008DE191E00E94390988E191E00E94390952
:101D10008AE2282E312C412C512C03E210E02FB7FF
:101D2000F89480918F0190919001A0919101B091D0
:101D300092012FBF20910A06382F321B232F30919A
:101D40000B06332309F43FC020930C0610920B06B8
:101D500080E090E0892B19F30E940000E0CF3E98CC
:101D60003F989DCF112331F0A981BA81149711F4C6
:101D70002E9A2F9881E00E94060420E148E56CEA43
:101D800075E089819A810E94150480E00E94060412
:101D90008FE090E00E94290789819A8101969A83B9
:101DA0008983499709F089CF112311F02F9A2D9833
:101DB00080E991E00E9429070E9427078EEF95E0B5
:101DC0000E94840C82CF30910906231748F42F5FBC
:101DD000231708F0BDCF81E083BF889513BEB8CF2D
:101DE00021E020930B0680930A06809105069091CE
:101DF0000606019690930606809305060E94F90355
:101E00001092100610920F0610920E0610920D06F8
:101E100080910706809308060E942E07809307068C
:101E2000809197018111A4C08091050690910606CA
:101E30006CE870E00E94421523E043E063E270E04A
:101E40008634910508F02AC349960E9478072AE053
:101E500042E06EE170E087E190E00E9478072AE0BE
:101E600042E06EE170E082E690E00E94780726E0B2
:101E700042E569E676E08FE090E00E941504B1E06B
:101E8000B09313068AE290E090930E0680930D06BD
:101E90008DE290E09093100680930F068FE591E01D
:101EA0000E94FC0884E190E090930E0680930D065A
:101EB00087E390E09093100680930F0687E691E009
:101EC0000E94FC0880919301909194010E9409095D
:101ED00080E00E9406048091080683FD49C080913D
:101EE000070683FF45C091E0909397018DE191E053
:101EF0000E94390988E191E00E94390980E090E070
:101F0000A0E2B1E48093000190930101A09302014B
:101F1000B093030180E090E0A0E2B2E4809304017A
:101F200090930501A0930601B093070180E090E033
:101F3000A0E8BFE380930C0190930D01A0930E01E4
:101F4000B0930F0110921001109211011092120122
:101F50001092130110929601109295010E94F903BC
:101F60001092100610920F0610920E0610920D0697
:101F700080919701833061F4809195019091960151
:101F80000196909396018093950181E0809397014B
:101F900080919701813009F005C2ACE3B0E0B093C5
:101FA0000E06A0930D068EE190E0909310068093AC
:101FB0000F0680919501909196010E9409098091E8
:101FC000190190911B01891728F420911A01820FA1
:101FD0008093190180911901981728F490911A01A2
:101FE000891B809319016091190170E0809118019B
:101FF00022E142E090E00E94780780911E019091DA
:102000002001891728F420911F01820F80931E015F
:1020100080911E01981728F490911F01891B8093CD
:102020001E0160911E0170E080911D0122E142E0DD
:1020300090E00E9478078091080687FD04C0909187
:10204000070697FD06C083FD10C08091070683FF39
:102050000CC080E090E0A0E2B0EC8093100190937F
:102060001101A0931201B093130180910C01909182
:102070000D01A0910E01B0910F0189839A83AB836A
:10208000BC832091000130910101409102015091E7
:102090000301BC01CD010E9477136B017C01C0924A
:1020A0000001D0920101E0920201F09203018091BF
:1020B000100190911101A0911201B09113018D8333
:1020C0009E83AF83B8872091040130910501409130
:1020D000060150910701BC01CD010E9477133B011D
:1020E0004C01609204017092050180920601909269
:1020F0000701909105069987A0910606AA8790FD91
:1021000016C02D813E814F815885609114017091D8
:10211000150180911601909117010E947713609329
:10212000100170931101809312019093130189851E
:102130009A8562E370E00E944215892B91F428EBA6
:102140003EE145E85FE369817A818B819C810E9451
:10215000D51460930C0170930D0180930E01909340
:102160000F0120E030E040EF52E4C701B6010E94C9
:10217000D01418160CF05AC0A0901E01B12C20E00B
:1021800030E040E450E4C401B3010E9477136B01D6
:102190007C01B5010B2C000C880B990B0E942014BC
:1021A0009B01AC01C701B6010E94D01418160CF0B7
:1021B0007CC1B5016E5E7F4F072E000C880B990B1A
:1021C0000E9420149B01AC01C401B3010E94E313DF
:1021D00087FF6BC1C0900C01D0900D01E0900E0103
:1021E000F0900F0120E030E0A901C701B6010E9484
:1021F000D014181624F4F7FAF094F7F8F094C0927B
:102200000C01D0920D01E0920E01F0920F010E949C
:10221000A512A20191010E9413136D5F7F4F8F4F92
:102220009F4F6093200183E08093970120E030E08E
:1022300040EC50E460910001709101018091020135
:10224000909103010E94E31387FF61C0C0900401D5
:10225000D0900501E0900601F0900701609019010F
:10226000712C20E030E040E450E4C701B6010E9448
:1022700077134B015C01B301072C000C880B990B01
:102280000E9420149B01AC01C501B4010E94D0142E
:1022900018160CF00CC1B3016E5E7F4F072E000CB8
:1022A000880B990B0E942014A70196010E94D0145C
:1022B00018160CF0FCC0C0900C01D0900D01E090FD
:1022C0000E01F0900F0120E030E0A901C701B60136
:1022D0000E94D014181624F0F7FAF094F7F8F0944E
:1022E000C0920C01D0920D01E0920E01F0920F010C
:1022F0000E94A512A20191010E9413136D5F7F4FEE
:102300008F4F9F4F60931B0183E080939701C09094
:102310000401D0900501E0900601F090070120E053
:1023200030E044E852E4C701B6010E94D014181608
:102330006CF420E030E04AE753E4C701B6010E94A4
:10234000E31387FF03C082E0809397016091080147
:102350007091090180910A0190910B010E94EF1385
:102360006983C701B6010E94E8136B016091000107
:102370007091010180910201909103010E94E81384
:10238000CB012981422FB6010E9478078CE390E0AF
:1023900090930E0680930D06ABE1B0E0B09310066B
:1023A000A0930F0680919701823009F073C00E94BC
:1023B000F9031092100610920F0610920E0610925A
:1023C0000D060E94A512A20191010E9413136D5FD8
:1023D0007F4F8F4F9F4F60931E010E94A512A20155
:1023E00091010E9413136D5F7F4F8F4F9F4F60933A
:1023F0001E01809195019091960120919301309159
:10240000940128173907BCF49093940180939301A9
:102410008EE190E090930E0680930D06AFE0B0E061
:10242000B0931006A0930F0681E08093130684E713
:1024300091E00E94FC0810930E0600930D06109385
:10244000100600930F06B1E0B093130680E891E008
:102450000E94FC0810930E0600930D0682E390E0A4
:102460009093100680930F0691E0909313068CE6EC
:1024700091E00E94FC0880919501909196010E9444
:10248000090980E00E94060488EB9BE00E9429076E
:102490001092970180E00E9406045ACCE5EAF0E031
:1024A000DF01A81BB90BCD01D0CC82E0BDCE82E00C
:1024B0002CCF8F929F92AF92BF92CF92DF92EF92EA
:1024C000FF92CF93DF93EC01688179818A819B81B0
:1024D000611571058105910521F464E279ED8BE5C3
:1024E00097E02DE133EF41E050E00E9413134901E2
:1024F0005A019B01AC01A7EAB1E40E9432136B01BF
:102500007C01ACEEB4EFA50194010E944013C60E0D
:10251000D71EE81EF91EF7FE06C081E0C81AD108D2
:10252000E10880E8F80AC882D982EA82FB82C70102
:10253000B6019F77DF91CF91FF90EF90DF90CF9022
:10254000BF90AF909F908F9008958F929F92AF927F
:10255000BF92CF92DF92EF92FF9260912E01709125
:102560002F01809130019091310161157105810534
:10257000910521F464E279ED8BE597E02DE133EFED
:1025800041E050E00E94131349015A019B01AC0144
:10259000A7EAB1E40E9432136B017C01ACEEB4EF08
:1025A000A50194010E944013C60ED71EE81EF91E15
:1025B000F7FE06C081E0C81AD108E10880E8F80AF1
:1025C000C0922E01D0922F01E0923001F0923101A1
:1025D000C701B6019F77FF90EF90DF90CF90BF903B
:1025E000AF909F908F90089560932E0170932F016C
:1025F00080933001909331010895F999FECF92BDF7
:1026000081BDF89A992780B50895262FF999FECFB4
:102610001FBA92BD81BD20BD0FB6F894FA9AF99AFF
:102620000FBE01960895052E97FB1EF400940E949C
:102630002A1357FD07D00E94451307FC03D04EF420
:102640000C942A1350954095309521953F4F4F4F4C
:102650005F4F089590958095709561957F4F8F4F4E
:102660009F4F08950E946713A59F900DB49F900DF2
:10267000A49F800D911D11240895B7FF0C9432136F
:102680000E943213821B930B0895A1E21A2EAA1BFB
:10269000BB1BFD010DC0AA1FBB1FEE1FFF1FA21712
:1026A000B307E407F50720F0A21BB30BE40BF50B0F
:1026B000661F771F881F991F1A9469F76095709598
:1026C000809590959B01AC01BD01CF010895A29F1B
:1026D000B001B39FC001A39F700D811D1124911DF6
:1026E000B29F700D811D1124911D08955058BB2774
:1026F000AA270E948E130C9496140E94881438F016
:102700000E948F1420F039F49F3F19F426F40C94A2
:1027100085140EF4E095E7FB0C947F14E92F0E94DA
:10272000A71458F3BA17620773078407950720F0B8
:1027300079F4A6F50C94C9140EF4E0950B2EBA2F7B
:10274000A02D0B01B90190010C01CA01A0011124B7
:10275000FF27591B99F0593F50F4503E68F11A1663
:10276000F040A22F232F342F4427585FF3CF4695F4
:1027700037952795A795F0405395C9F77EF41F1616
:10278000BA0B620B730B840BBAF09150A1F0FF0FE0
:10279000BB1F661F771F881FC2F70EC0BA0F621FCC
:1027A000731F841F48F4879577956795B795F795BC
:1027B0009E3F08F0B0CF9395880F08F09927EE0F51
:1027C0009795879508950E945B1408F481E0089519
:1027D0000E94EF136894B1110C94CA1408950E94DA
:1027E000AF1488F09F5798F0B92F9927B751B0F0E0
:1027F000E1F0660F771F881F991F1AF0BA95C9F785
:1028000014C0B13091F00E94C914B1E008950C9445
:10281000C914672F782F8827B85F39F0B93FCCF3F8
:10282000869577956795B395D9F73EF49095809501
:10283000709561957F4F8F4F9F4F0895E89409C021
:1028400097FB3EF490958095709561957F4F8F4FE3
:102850009F4F9923A9F0F92F96E9BB279395F695F9
:10286000879577956795B795F111F8CFFAF4BB0F77
:1028700011F460FF1BC06F5F7F4F8F4F9F4F16C0DB
:10288000882311F096E911C0772321F09EE8872F65
:10289000762F05C0662371F096E8862F70E060E021
:1028A0002AF09A95660F771F881FDAF7880F96959A
:1028B000879597F90895990F0008550FAA0BE0E83E
:1028C000FEEF16161706E807F907C0F012161306F2
:1028D000E407F50798F0621B730B840B950B39F432
:1028E0000A2661F0232B242B252B21F408950A2698
:1028F00009F4A140A6958FEF811D811D089597F9D8
:102900009F6780E870E060E008959FEF80EC089595
:1029100000240A94161617061806090608950024BE
:102920000A9412161306140605060895092E039438
:10293000000C11F4882352F0BB0F40F4BF2B11F4AC
:1029400060FF04C06F5F7F4F8F4F9F4F089557FD0B
:102950009058440F551F59F05F3F71F04795880F0D
:1029600097FB991F61F09F3F79F0879508951216A4
:1029700013061406551FF2CF4695F1DF08C0161650
:1029800017061806991FF1CF869571056105089401
:102990000895E894BB2766277727CB0197F9089518
:1029A0000E945B1408F48FEF08950E94E8140C94C1
:1029B00096140E94881438F00E948F1420F09523FA
:1029C00011F00C947F140C94851411240C94CA14E7
:1029D0000E94A71470F3959FC1F3950F50E0551F07
:1029E000629FF001729FBB27F00DB11D639FAA2764
:1029F000F00DB11DAA1F649F6627B00DA11D661FB3
:102A0000829F2227B00DA11D621F739FB00DA11DD3
:102A1000621F839FA00D611D221F749F3327A00D8D
:102A2000611D231F849F600D211D822F762F6A2F29
:102A300011249F5750409AF0F1F088234AF0EE0F8E
:102A4000FF1FBB1F661F771F881F91505040A9F7BB
:102A50009E3F510580F00C947F140C94CA145F3F84
:102A6000E4F3983ED4F3869577956795B795F795F7
:102A7000E7959F5FC1F7FE2B880F911D969587956F
:102A800097F90895AA1BBB1B51E107C0AA1FBB1FE2
:102A9000A617B70710F0A61BB70B881F991F5A95EA
:102AA000A9F780959095BC01CD010895EE0FFF1F09
:102AB0000590F491E02D099481E090E0F8940C9455
:062AC0006115F894FFCF40
:102AC600000020410000A041000040400000803F7F
:102AD600000000009A99993E0000010000000001E4
:102AE6000000FFFFFFFF00E1000000000000010002
:102AF600000000C18081000000000000000A05A25D
:102B0600062B05200571052F054D0500000000A6C2
:102B1600071D06AB08AA08840CFCFF0000C60C5073
:102B260072657373204100486967682053636F724A
:102B3600653A20004E6577205265636F7264210006
:0A2B460047616D65204F766572004F
:00000001FF
